:1000000012C02CC02BC02AC029C028C027C026C0BF
:1000100025C063C2F6C26BC121C020C01DCA1EC06C
:100020001DC01CC01BC011241FBECFE5D4E0DEBF25
:10003000CDBF11E0A0E6B0E0E2ECF9E102C005902E
:100040000D92A033B107D9F711E0A0E3B1E001C0F0
:100050001D92AE3BB107E1F715D0B1CCD1CFDF9304
:10006000CF93CDB7DEB7E1E3F0E082E88083E7E34A
:10007000F0E080E18083E8E3F0E088E28083CF91E4
:10008000DF9108950F931F93DF93CF9300D0CDB7E7
:10009000DEB7E5DF13D293D0D1D98BD201E510E0E2
:1000A00084E090E059D0F801808380E090E075D042
:1000B00090938C0180938B0182E090E06ED09A83C4
:1000C000898389E78093630189819A8182339105CD
:1000D00019F489E78093630189819A8184369105B7
:1000E00019F482EF80936301A2E3B0E0E2E3F0E071
:1000F000808180688C93789480E690E0BED0EED0CA
:1001000085E580937C0185E480937D0185E690E020
:100110009093800180937F018EEF90E09093820115
:100120008093810151D280938A0180913101813085
:1001300029F41092310180E090E0E0D98091320101
:10014000813011F41092320180913A01813051F7DF
:1001500010923A0191D2E6CFDF93CF9300D00F9265
:10016000CDB7DEB79B838A83ECE3F0E08081882FF4
:1001700090E0827090700097B9F7EEE3F0E08A812A
:100180009B8191838083E09A8DB3898389810F90CD
:100190000F900F90CF91DF910895DF93CF9300D010
:1001A000CDB7DEB79A83898389819A812CEA30E0C2
:1001B000B90120DB0F900F90CF91DF910895DF936D
:1001C000CF93CDB7DEB7E9E2F0E080E18083E0E4F1
:1001D000F0E01082A8E3B0E0E8E3F0E08081816025
:1001E0008C93EAE2F0E088E98083E0E4F0E086E8DE
:1001F0008083EBE2F0E082EC8083CF91DF91089581
:10020000DF93CF930F92CDB7DEB78983EBE2F0E0B7
:100210008081882F90E0807290700097B9F3ECE2B3
:10022000F0E0898180830F90CF91DF910895DF9373
:10023000CF9300D000D0CDB7DEB79B838A836C8389
:100240008C81882399F019820DC08981282F30E094
:100250008A819B81FC01E20FF31F8081D1DF8981BC
:100260008F5F898399818C81891778F70F900F9020
:100270000F900F90CF91DF910895DF93CF9300D02F
:1002800000D00F92CDB7DEB79D838C838C819D818A
:10029000A8DA9A8389831B820FC08B81282F33278A
:1002A00027FD30958C819D81FC01E20FF31F808139
:1002B000A7DF8B818F5F8B838B81282F332727FDCF
:1002C000309589819A812817390738F30F900F905C
:1002D0000F900F900F90CF91DF910895DF93CF9300
:1002E000CDB7DEB78EE38CDFCF91DF9108951F92FB
:1002F0000F920FB60F9211242F933F934F935F935A
:100300006F937F938F939F93AF93BF93EF93FF93DD
:10031000DF93CF9300D000D00F92CDB7DEB7ECE2E1
:10032000F0E0808180939C0180919C0169DF809145
:100330009C018D3079F03091BB01832F90E02091AA
:100340009C01FC01EB5BFE4F2083832F8F5F80932A
:10035000BB019CC08091BB01882F90E020919C0143
:10036000FC01EB5BFE4F20831A8219821092370149
:1003700010923801109239011B827DC08A81282F8A
:1003800030E03D832C838C819D818130910569F122
:100390002C813D812230310509F449C08C819D8139
:1003A000009709F065C08B81882F90E0FC01EB5B22
:1003B000FE4F80818032A9F08981282F30E08B8127
:1003C000882F90E0FC01EB5BFE4F8081F901EF5438
:1003D000FE4F808389818093370189818F5F898374
:1003E00047C081E08A83198243C08B81882F90E0C7
:1003F000FC01EB5BFE4F80818032A9F08981282FC0
:1004000030E08B81882F90E0FC01EB5BFE4F808118
:10041000F901E955FE4F80838981809338018981F4
:100420008F5F898325C082E08A83198221C08B81F6
:10043000882F90E0FC01EB5BFE4F80818032A9F0B9
:100440008981282F30E08B81882F90E0FC01EB5BC5
:10045000FE4F8081F901E356FE4F808389818093AE
:10046000390189818F5F898303C083E08A83198280
:100470008B818F5F8B839091BB018B81981708F0E4
:100480007DCF81E080933A011092BB010F900F90D5
:100490000F900F900F90CF91DF91FF91EF91BF914F
:1004A000AF919F918F917F916F915F914F913F910C
:1004B0002F910F900FBE0F901F901895DF93CF9341
:1004C000CDB7DEB7E3E5F0E082E08083E9E5F0E078
:1004D00081E08083CF91DF9108951F920F920FB634
:1004E0000F9211248F93DF93CF9300D0CDB7DEB757
:1004F00080913E018A8319828A81843011F481E0DF
:1005000089838A818F5F80933E018981882329F0C6
:1005100081E08093350110923E0180918D018F5FC3
:1005200080938D0180918D018732C9F581E08093A0
:10053000330110928D0180913D018F5F80933D01C9
:1005400080913D01853029F410923D0181E0809336
:10055000340180913B018F5F80933B0180913B018F
:10056000843641F410923B0181E08093300181E0B8
:100570008093320180913B01823319F481E08093B2
:10058000320180913C018F5F80933C0180913C015E
:100590008A3029F410923C0181E0809331010F9060
:1005A0000F90CF91DF918F910F900FBE0F901F9002
:1005B0001895DF93CF93CDB7DEB7EDE2F0E080EC96
:1005C0008083CF91DF910895DF93CF930F92CDB7C2
:1005D000DEB7E6E3F0E08081882F90E084709070D1
:1005E000009749F080913F01882311F010923F015C
:1005F00081E0898301C0198289810F90CF91DF91B9
:1006000008951F920F920FB60F9211242F933F93CC
:100610004F938F939F93AF93BF93EF93FF93DF938A
:10062000CF930F92CDB7DEB7AFE2B0E02091750067
:100630003091760040913F01842F90E0F901E80F5E
:10064000F91F80818C93842F8F5F80933F01EFE2AD
:10065000F0E0808189830F90CF91DF91FF91EF913E
:10066000BF91AF919F918F914F913F912F910F909B
:100670000FBE0F901F901895DF93CF93CDB7DEB7C5
:10068000C55FD0400FB6F894DEBF0FBECDBF9E0150
:10069000235F3F4FC753DF4F39832883C95CD04066
:1006A00083EA90E0C553DF4F99838883CB5CD040C9
:1006B00098E0C353DF4F9883CD5CD040C553DF4FE4
:1006C000E881F981CB5CD0400080C553DF4F2881A1
:1006D0003981CB5CD0402F5F3F4FC553DF4F39830B
:1006E0002883CB5CD040C753DF4FE881F981C95CD8
:1006F000D0400082C753DF4F28813981C95CD04088
:100700002F5F3F4FC753DF4F39832883C95CD040E9
:10071000C353DF4F3881CD5CD0403150C353DF4FDE
:100720003883CD5CD040C353DF4F8881CD5CD0404F
:10073000882321F6FE017596C253DF4FF983E883C3
:10074000CE5CD0402BEA30E0C053DF4F39832883A2
:10075000C05DD0403FE0CE52DF4F3883C25DD04015
:10076000C053DF4FE881F981C05DD0400080C053A5
:10077000DF4F28813981C05DD0402F5F3F4FC0538C
:10078000DF4F39832883C05DD040C253DF4FE881FB
:10079000F981CE5CD0400082C253DF4F288139817D
:1007A000CE5CD0402F5F3F4FC253DF4F3983288349
:1007B000CE5CD040CE52DF4F3881C25DD040315048
:1007C000CE52DF4F3883C25DD040CE52DF4F88819A
:1007D000C25DD040882321F6FE01B496CD52DF4F92
:1007E000F983E883C35DD0402AEB30E0CB52DF4F82
:1007F00039832883C55DD0403DE0C952DF4F38833F
:10080000C75DD040CB52DF4FE881F981C55DD04054
:100810000080CB52DF4F28813981C55DD0402F5FEA
:100820003F4FCB52DF4F39832883C55DD040CD5237
:10083000DF4FE881F981C35DD0400082CD52DF4FA8
:1008400028813981C35DD0402F5F3F4FCD52DF4FAC
:1008500039832883C35DD040C952DF4F3881C75DDB
:10086000D0403150C952DF4F3883C75DD040C952A4
:10087000DF4F8881C75DD040882321F6FE01F196C5
:10088000C852DF4FF983E883C85DD04027EC30E0E1
:10089000C652DF4F39832883CA5DD04038E0C45246
:1008A000DF4F3883CC5DD040C652DF4FE881F981FD
:1008B000CA5DD0400080C652DF4F28813981CA5DB1
:1008C000D0402F5F3F4FC652DF4F39832883CA5D28
:1008D000D040C852DF4FE881F981C85DD040008226
:1008E000C852DF4F28813981C85DD0402F5F3F4F0C
:1008F000C852DF4F39832883C85DD040C452DF4FD0
:100900003881CC5DD0403150C452DF4F3883CC5D4C
:10091000D040C452DF4F8881CC5DD040882321F67F
:10092000FE01F996C352DF4FF983E883CD5DD040D5
:100930002FEC30E0C152DF4F39832883CF5DD040A8
:100940003DE0CF51DF4F3883C15ED040C152DF4F11
:10095000E881F981CF5DD0400080C152DF4F28810E
:100960003981CF5DD0402F5F3F4FC152DF4F398378
:100970002883CF5DD040C352DF4FE881F981CD5D40
:10098000D0400082C352DF4F28813981CD5DD040F5
:100990002F5F3F4FC352DF4F39832883CD5DD04057
:1009A000CF51DF4F3881C15ED0403150CF51DF4F42
:1009B0003883C15ED040CF51DF4F8881C15ED040C7
:1009C000882321F6CE018A5B9F4FCE51DF4F99835A
:1009D0008883C25ED040ECEDF0E0CC51DF4FF9836C
:1009E000E883C45ED040F4E1CA51DF4FF883C65EAD
:1009F000D040CC51DF4FE881F981C45ED040008007
:100A0000CC51DF4F28813981C45ED0402F5F3F4FEA
:100A1000CC51DF4F39832883C45ED040CE51DF4FA5
:100A2000E881F981C25ED0400082CE51DF4F28813B
:100A30003981C25ED0402F5F3F4FCE51DF4F3983A7
:100A40002883C25ED040CA51DF4F3881C65ED04095
:100A50003150CA51DF4F3883C65ED040CA51DF4F94
:100A60008881C65ED040882321F6CE01865A9F4FEA
:100A7000C951DF4F99838883C75ED040E0EFF0E033
:100A8000C751DF4FF983E883C95ED040F5E1C55116
:100A9000DF4FF883CB5ED040C751DF4FE881F9814B
:100AA000C95ED0400080C751DF4F28813981C95EBF
:100AB000D0402F5F3F4FC751DF4F39832883C95E36
:100AC000D040C951DF4FE881F981C75ED040008234
:100AD000C951DF4F28813981C75ED0402F5F3F4F1A
:100AE000C951DF4F39832883C75ED040C551DF4FDE
:100AF0003881CB5ED0403150C551DF4F3883CB5E5B
:100B0000D040C551DF4F8881CB5ED040882321F68D
:100B1000CE0181599F4FC451DF4F99838883CC5EAA
:100B2000D040E5E0F1E0C251DF4FF983E883CE5ECB
:100B3000D040FBE0C051DF4FF883C05FD040C251CE
:100B4000DF4FE881F981CE5ED0400080C251DF4F97
:100B500028813981CE5ED0402F5F3F4FC251DF4F99
:100B600039832883CE5ED040C451DF4FE881F981BC
:100B7000CC5ED0400082C451DF4F28813981CC5EE9
:100B8000D0402F5F3F4FC451DF4F39832883CC5E65
:100B9000D040C051DF4F3881C05FD0403150C0518C
:100BA000DF4F3883C05FD040C051DF4F8881C05FC6
:100BB000D040882321F6CE0186589F4FCF50DF4F7B
:100BC00099838883C15FD040E0E1F1E0CD50DF4FF1
:100BD000F983E883C35FD040F7E1CB50DF4FF88360
:100BE000C55FD040CD50DF4FE881F981C35FD04071
:100BF0000080CD50DF4F28813981C35FD0402F5F07
:100C00003F4FCD50DF4F39832883C35FD040CF5053
:100C1000DF4FE881F981C15FD0400082CF50DF4FC4
:100C200028813981C15FD0402F5F3F4FCF50DF4FC8
:100C300039832883C15FD040CB50DF4F3881C55FF7
:100C4000D0403150CB50DF4F3883C55FD040CB50C0
:100C5000DF4F8881C55FD040882321F68091B101A4
:100C6000C853DF4F1882C85CD040883631F491E019
:100C7000C853DF4F9883C85CD0408091B201C953FC
:100C8000DF4F1882C75CD040853631F4E1E0C953AC
:100C9000DF4FE883C75CD040C853DF4F8881C85C12
:100CA000D040C953DF4FF881C75CD0408F23282F35
:100CB00030E0CB53DF4F39832883C55CD04080912F
:100CC000B301CD53DF4F19821882C35CD0408C36FC
:100CD00041F481E090E0CD53DF4F99838883C35C7A
:100CE000D040CB53DF4FE881F981C55CD040CD5374
:100CF000DF4F28813981C35CD040E223F323CF53F7
:100D0000DF4FF983E883C15CD0408091B401C154C6
:100D1000DF4F19821882CF5BD040803741F481E0E9
:100D200090E0C154DF4F99838883CF5BD040CF538D
:100D3000DF4F88819981C15CD040C154DF4FE88189
:100D4000F981CF5BD0408E239F230097D9F0CE014D
:100D50000D9693DACE01459690DACE0184968DDA1F
:100D6000CE01C1968ADACE01C99687DACE018A5BB6
:100D70009F4F83DACE01865A9F4F7FDACE01815989
:100D80009F4F7BDA8091B101C254DF4F1882CE5B56
:100D9000D040833731F4F1E0C254DF4FF883CE5BAB
:100DA000D0408091B201C354DF4F1882CD5BD04058
:100DB000883631F421E0C354DF4F2883CD5BD04027
:100DC000C254DF4F8881CE5BD040C354DF4F38819F
:100DD000CD5BD0408323E82FF0E0C554DF4FF9838B
:100DE000E883CB5BD0408091B301C754DF4F1982B9
:100DF0001882C95BD0408F3641F421E030E0C754FF
:100E0000DF4F39832883C95BD040C554DF4F8881C9
:100E10009981CB5BD040C754DF4FE881F981C95B32
:100E2000D0408E239F23C954DF4F99838883C75BAB
:100E3000D0408091B401CB54DF4F19821882C55B3A
:100E4000D040873741F421E030E0CB54DF4F398385
:100E50002883C55BD040C954DF4F88819981C75B27
:100E6000D040CB54DF4FE881F981C55BD0408E2361
:100E70009F23009709F49FC08091A701CC54DF4FB6
:100E80001882C45BD040863731F4F1E0CC54DF4F98
:100E9000F883C45BD0408091A801CD54DF4F188205
:100EA000C35BD040853631F421E0CD54DF4F288339
:100EB000C35BD040CC54DF4F8881C45BD040CD545D
:100EC000DF4F3881C35BD0408323882321F0CE01DC
:100ED00086589F4FD2D98091A701CE54DF4F1882F8
:100EE000C25BD040833731F481E0CE54DF4F88833A
:100EF000C25BD0408091A801CF54DF4F1882C15B04
:100F0000D040843731F491E0CF54DF4F9883C15BF8
:100F1000D040CE54DF4F8881C25BD040CF54DF4FEA
:100F2000E881C15BD0408E23882319F081E0809353
:100F300036018091A701C055DF4F1882C05BD040B9
:100F4000833731F4F1E0C055DF4FF883C05BD04008
:100F50008091A801C155DF4F1882CF5AD040863604
:100F600031F421E0C155DF4F2883CF5AD040C0551E
:100F7000DF4F8881C05BD040C155DF4F3881CF5AE9
:100F8000D04083238823B9F082E090E0D5D19A83C2
:100F9000898389819A819E012D5F3F4FB9014AE083
:100FA00050E053D487E790E068D9CE01039665D925
:100FB00087E890E062D98091B101C255DF4F188275
:100FC000CE5AD040833731F481E0C255DF4F888359
:100FD000CE5AD0408091B201C355DF4F1882CD5A0E
:100FE000D040843731F491E0C355DF4F9883CD5A18
:100FF000D040C255DF4F8881CE5AD040C355DF4F15
:10100000E881CD5AD0408E23282F30E0C555DF4FE0
:1010100039832883CB5AD0408091B301C755DF4F25
:1010200019821882C95AD0408F3641F481E090E08D
:10103000C755DF4F99838883C95AD040C555DF4FC4
:10104000E881F981CB5AD040C755DF4F28813981DB
:10105000C95AD040E223F323C955DF4FF983E8830F
:10106000C75AD0408091B401CB55DF4F1982188206
:10107000C55AD040803741F481E090E0CB55DF4F36
:1010800099838883C55AD040C955DF4F888199819B
:10109000C75AD040CB55DF4FE881F981C55AD040BF
:1010A0008E239F23009711F0109236018091B10199
:1010B000CC55DF4F1882C45AD040833731F4F1E069
:1010C000CC55DF4FF883C45AD0408091B201CD5542
:1010D000DF4F1882C35AD040853631F421E0CD5518
:1010E000DF4F2883C35AD040CC55DF4F8881C45A84
:1010F000D040CD55DF4F3881C35AD0408323E82FED
:10110000F0E0CF55DF4FF983E883C15AD04080919A
:10111000B301C156DF4F19821882CF59D0408437AE
:1011200041F421E030E0C156DF4F39832883CF59A5
:10113000D040CF55DF4F88819981C15AD040C156E8
:10114000DF4FE881F981CF59D0408E239F2300974C
:1011500009F46DC08091A701C256DF4F1882CE59A5
:10116000D040833631F4F1E0C256DF4FF883CE59D8
:10117000D0408091A801C356DF4F1882CD59D0408E
:101180008A3731F421E0C356DF4F2883CD59D04050
:10119000C256DF4F8881CE59D040C356DF4F3881C9
:1011A000CD59D0408323882341F08DE991E0FCD2D2
:1011B00090938C0180938B01A8D28091A701C45693
:1011C000DF4F1882CC59D040833731F481E0C456C8
:1011D000DF4F8883CC59D0408091A801C556DF4F9E
:1011E0001882CB59D040863631F491E0C556DF4F96
:1011F0009883CB59D040C456DF4F8881CC59D0401A
:10120000C556DF4FE881CB59D0408E23882379F033
:101210008DE991E0C9D29A83898382E090E02981A7
:101220003A81B901BCD089E890E027D8F8D0809104
:10123000B101C656DF4F1882CA59D040823731F407
:10124000F1E0C656DF4FF883CA59D0408091B20111
:10125000C756DF4F1882C959D040853631F421E096
:10126000C756DF4F2883C959D040C656DF4F888103
:10127000CA59D040C756DF4F3881C959D04083235F
:10128000E82FF0E0C956DF4FF983E883C759D04013
:101290008091B301CB56DF4F19821882C559D040D7
:1012A000833741F421E030E0CB56DF4F3983288388
:1012B000C559D040C956DF4F88819981C759D04060
:1012C000CB56DF4FE881F981C559D0408E239F234B
:1012D000CD56DF4F99838883C359D0408091B401A4
:1012E000CF56DF4F19821882C159D040853641F45C
:1012F00021E030E0CF56DF4F39832883C159D040F9
:10130000CD56DF4F88819981C359D040CF56DF4FEA
:10131000E881F981C159D0408E239F23009709F0BD
:101320007ED0DCD7CB50DF4F0FB6F894DEBF0FBEB8
:10133000CDBFCF91DF910895DF93CF9300D0CDB78C
:10134000DEB79A83898389819A812EEA39E0B901CF
:1013500051D20F900F90CF91DF910895DF93CF93EB
:1013600000D00F92CDB7DEB79B838A83ECE3F0E029
:101370008081882F90E0827090700097B9F7EEE33B
:10138000F0E08A819B8191838083E09A8DB3898389
:1013900089810F900F900F90CF91DF910895DF9387
:1013A000CF9300D000D0CDB7DEB79A8389837C83FA
:1013B0006B8389819A812B813C8148EE59E0B90188
:1013C0002FD20F900F900F900F90CF91DF91089533
:1013D000DF93CF9300D00F92CDB7DEB79A83898386
:1013E0006B83ECE3F0E08081882F90E08270907056
:1013F0000097B9F7EEE3F0E089819A8191838083C9
:10140000EDE3F0E08B8180830FB6F894E29AE19AE5
:101410000FBE0F900F900F90CF91DF910895DF9343
:10142000CF93CDB7DEB7F89488E190E028E00FB60F
:10143000F894A89581BD0FBE21BDFFCFDF93CF9358
:10144000CDB7DEB7E7E2F0E01082E6E2F0E08FE849
:101450008083CF91DF9108951F920F920FB60F9264
:1014600011242F933F934F935F938F939F93EF9309
:10147000FF93DF93CF93CDB7DEB7E6E2F0E01082C3
:1014800080912701482F50E0E4E2F0E080819181D3
:101490009C01CA01880F991FFC01E257FE4F31835E
:1014A000208380912701482F50E0882F90E0880FFB
:1014B000991FFC01E257FE4F2081318180918B0101
:1014C00090918C01281B390BCA01880F991FFC01D0
:1014D000E257FE4F3183208381E080934001CF911A
:1014E000DF91FF91EF919F918F915F914F913F918C
:1014F0002F910F900FBE0F901F901895DF93CF93F1
:10150000CDB7DEB76C970FB6F894DEBF0FBECDBF78
:101510008C8F809127018F5F809327018091270115
:10152000853008F4E2C0109227011F8218861986C0
:101530001A861B862BC08B85992787FD9095880F6F
:10154000991FFC01E257FE4F208131818091630198
:10155000882F90E0AC01249FC001259F900D349FFF
:10156000900D11249C01442737FD4095542F8F8105
:101570009885A985BA85820F931FA41FB51F8F83F5
:101580009887A987BA878B858F5F8B878B858530F6
:1015900094F28F819885A985BA8525E030E040E0F6
:1015A00050E0BC01CD01BAD1DA01C9018B839C8323
:1015B000AD83BE83209141013091420140914301AE
:1015C000509144018F819885A985BA85820F931F18
:1015D000A41FB51F8093410190934201A093430142
:1015E000B09344018091410190914201A091430147
:1015F000B091440120EA3CE840E050E0BC01CD015C
:101600008DD1DA01C9019A838983DED78823E9F372
:1016100085E580937C018B819C81AD81BE8128EE24
:1016200033E040E050E0BC01CD0178D1DA01C901DE
:1016300080937D018B819C81AD81BE8128EE33E05A
:1016400040E050E0BC01CD0169D1DC01CB0124E6D2
:1016500030E040E050E0BC01CD0160D1DA01C901C9
:1016600080937E0185E690E09093800180937F01D6
:1016700089819A81909382018093810180913601C2
:10168000813099F580918E0190918F019E01245FA8
:101690003F4FB9014AE050E0D8D0CE010C96EDD5CD
:1016A00088E291E0EAD58B819C81AD81BE819E016B
:1016B000245F3F4FBC01CD01A9012AE030E0E4D016
:1016C000CE010C96DAD588E291E0D7D589819A814E
:1016D0009E01245F3F4FB9014AE050E0B6D0CE01F1
:1016E0000C96CBD58DE291E0C8D5E7E2F0E0108210
:1016F000E6E2F0E08FEC80836C960FB6F894DEBFE4
:101700000FBECDBFCF91DF910895DF93CF93CDB7BB
:10171000DEB780E090E020918B0130918C01B9011F
:1017200003D0CF91DF910895DF93CF9300D000D005
:10173000CDB7DEB79A8389837C836B8389819A8155
:101740002B813C814DEA5BE0B9016AD00F900F908C
:101750000F900F90CF91DF910895DF93CF9300D03A
:101760000F92CDB7DEB79A8389836B83ECE3F0E009
:101770008081882F90E0827090700097B9F7EEE337
:10178000F0E089819A8191838083EDE3F0E08B81A1
:1017900080830FB6F894E29AE19A0FBE0F900F90F3
:1017A0000F90CF91DF910895FC0188279927E89445
:1017B00021912032E9F3293010F02E30C8F32B327A
:1017C00039F02D3231F4689403C090D0820F911D0E
:1017D000219120532A30C8F31EF4909581959F4F94
:1017E0000895FC0101900020E9F7809590958E0FF7
:1017F0009F1F0895DF92EF92FF920F931F937B013B
:101800008C01FB010995D82EC8010196F7010995B5
:10181000982F8D2D1F910F91FF90EF90DF900895DD
:10182000DF92EF92FF920F931F93D72E7A018C01D4
:10183000FA010995C80101966D2DF70109951F91CF
:101840000F91FF90EF90DF900895FB019F01E894C6
:101850004230BCF04532ACF44A3029F497FB1EF418
:10186000909581959F4F642F772795D0805D8A331F
:101870000CF0895D8193CB010097A9F716F45DE226
:1018800051931082C9013AC0FA01CF93FF93EF93AD
:1018900022303CF125322CF5C22FE894CA3049F4AD
:1018A00097FB3EF490958095709561957F4F8F4F93
:1018B0009F4F2C2F332744275527FF93EF9349D071
:1018C000EF91FF91605D6A330CF0695D6193B9013E
:1018D000CA01605070408040904059F716F4CDE244
:1018E000C19310828F919F91CF9108C07AE0979F0A
:1018F000902D879F802D910D11240895DC01FC010E
:10190000672F71917723E1F7329704C07C916D9333
:1019100070836291AE17BF07C8F3089597FB092E35
:1019200005260ED057FD04D014D00AD0001C38F480
:1019300050954095309521953F4F4F4F5F4F0895FB
:10194000F6F790958095709561957F4F8F4F9F4FDB
:101950000895A1E21A2EAA1BBB1BFD010DC0AA1FF0
:10196000BB1FEE1FFF1FA217B307E407F50720F008
:10197000A21BB30BE40BF50B661F771F881F991F83
:101980001A9469F760957095809590959B01AC01CC
:10199000BD01CF010895AA1BBB1B51E107C0AA1FBF
:1019A000BB1FA617B70710F0A61BB70B881F991F00
:1019B0005A95A9F780959095BC01CD010895F894AA
:0219C000FFCF57
:1019C2004550492D532056657273696F6E20302E33
:1019D200312E360D007C0153656E736F72204D619E
:1019E200782041203D20000D000D3E526573657444
:1019F2002041544D454741380D2E2E2E0D2E2E2EB0
:101A02002E0D0068656C70200D000073686F7720E2
:101A120076657273696F6E0D000073686F7720656B
:101A220072726F720D000072657365740D0000733F
:101A3200686F77207374726F6D0D00007365742088
:101A4200637A202863616C5F7A65726F290D0000EA
:101A520073657420736620283530202F2031303092
:101A62002029200D0073686F7720736620200D00F7
:101A72004550492D5374726F6D205665722E3A206F
:101A8200302E302E310D000520202000000D0000E8
:00000001FF
